:1000000003C0189518951895BA9A0CEF08BB0FE71E
:1000100001BBD8EE10E020E533EC40E050E060E0BA
:1000200033C0A9E0B0E0C0E0B5D193E101E000C089
:1000300000C000C0000076E134D14599FBCF7A952D
:10004000D9F700002ED1C29872E100C02AD17A956A
:10005000E1F7C29A74EB25D100C080E000C021D145
:100060008A95E1F77A95D9F700001BD19A9561F04E
:100070000A9531F0A12FB22FC32F142F252F362F21
:100080004A2F5B2F6C2FD3CF1AD1D7FF45C0D03862
:10009000E9F3D3FF34C1D83E19F0D83BB9F7D9C042
:1000A000A03009F4A3E0A03C21F0A7FD04C0AA0FF2
:1000B00007C0A0EE05C0A595AF7BA03809F4A3E06A
:1000C0000A2F009502BB91E0B5CFD83D09F4BFC01F
:1000D0001BE440E02FED50E03DEB61E0A0E0B0E537
:1000E000C3EC82C0D83D09F4AAC01EE540E027E178
:1000F00051E03DE262E0A0E0BAE6C8E175C0D83D5B
:1001000009F4A1C018E840E025E951E039E263E0D4
:10011000A9EEB2E8C3E268C035D1740F851F961FFF
:10012000D03761F1D83669F1D83549F3D833B1F118
:10013000D036C1F2D035F9F1D03309F1D83901F117
:10014000A4E7B1ECC1E1B5D0D0F0AEE8B3EBC5E1C6
:10015000B0D088F1ABEDB6EECBE1ABD018F2A7EAA8
:10016000B7EFC1E2A6D0D0F0AFECB3E3C5E2A1D0C7
:1001700030F2ABEABAE1C1E49CD018F0A6CF28C0B7
:100180000DC1D83D09F461C015E940E02DEB51E007
:100190003AE763E0A0E0B0E1C7E226C0D83D09F449
:1001A00050C01CE740E023E751E036EE62E0A5E5F1
:1001B000BDE8C0E219C0D83D09F43FC01BE440E0EF
:1001C0002FED50E03DEB61E0A0E0B8E8C3E10CC0EA
:1001D000D83D09F42FC01FE340E02AEB50E033E79D
:1001E00061E0ABEAB6E4C0E164D088F07A1B8B0B27
:1001F0009C0BA12FB42FC0E05CD018F1A22FB52F1B
:1002000058D008F1A32FB62F54D0F8F020C0A71B68
:10021000B80BC90B7A2F8B2F9C2FA12FB42FC0E0C6
:1002200048D078F0A22FB52F44D048F0A32FB62F96
:1002300040D018F00FE302BBF4CE0FE5FCCF0FE681
:10024000FACF07E7F8CF0BE7F6CF0DE7F4CF0EE7CD
:10025000F2CF98D09BD02DD020F0741B850B960B3D
:1002600006C0742F852F962F711B820B930BA1E074
:10027000B5E0C0E01ED058F3A1E0BFE01AD028F3EB
:10028000A1E0BEE116D0F8F2A1E0B2E312D0C8F2CC
:10029000A1E0B4E60ED098F2A1E0B8EC0AD068F282
:1002A000C9CF0000439521F4539509F4639508954F
:1002B000FECF9C17E9F78B1709F47A17089506B358
:1002C000087F083F09F0D02F0895EBDF1AE92DE6EB
:1002D00030E00FE302BB56D096958795779541E0C5
:1002E00050E060E01BD00FE702BB4CD017D0C298A3
:1002F00002E100C0D6DF0A95E1F7C29AE0DFD03F05
:1003000099F0D03EC1F0D03DE9F0D03B09F1D03CAE
:1003100031F1D03A59F1D039C1F283CE37D0C9DFAB
:1003200010F0BFDFFBCF089504E028D01EEB23E2DE
:1003300035E00EE7CFCF07E020D01CE127E031E029
:100340000DE7C8CFAEDF10E32FEE30E00BE7C2CFF2
:1003500005E014D010E42BED30E007E7BBCF03E05D
:100360000CD01DE624EA30E00FE6B4CF02E006D060
:1003700018E823E830E00FE5ADCF000000000A9553
:10038000F1F70895712F822F932F0895A42FB52F81
:10039000C62F08951A2F2B2F3C2F08950FE01EC053
:1003A0008EDFD037B9F0D03FB9F0D83679F0D83EEB
:1003B00079F0D83539F0D83D39F0D83189F70CEFDC
:1003C00002BB2FCE072F0AC0072F07C0082F06C079
:1003D000082F03C0092F02C0092F02950F70009546
:0403E00002BBDECFAF
:00000001FF
